:10000000B401BD28A70087130713071383168713AE
:1000100007130713F030870583122708B4182E281A
:100020003A30A100983097203330A6004320133097
:10003000A10088309720432064309620432064300C
:1000400096202230A600432028302D200C302D2071
:1000500006302D20B41427082E283414A600341C92
:100060003C280713033C031C412841200730A10012
:10007000D0309720031408003414FE3C0319B8282C
:100080000717A60E341C34108717F0308705260892
:100090000F3987048713A60E341843283230962070
:1000A0000314080064006820031852287920A8016E
:1000B0000830A3007A2068200318A80AAB1EA80104
:1000C000A20CA30B5A28AB1AA2137A20220808000C
:1000D00038088400360884178004841300052B1B1D
:1000E0003606FF3E080029080319B828B320A903E3
:1000F000732835172B081F39FF3EA1002A08F53E4B
:100100000318A10A351F97283513A0000230AE202E
:100110009728A301A200FF30A207031CA307031C1A
:10012000B8280330A100DF3097208B28A101E83EDA
:10013000A000A109FC30031CA028A00703189D28DB
:10014000A0076400A10F9D282018A628A01CAA289B
:100150000000AA2808000310A10CA00CFF3E031801
:10016000AB282008B828840031088A0030088200B3
:10017000831303138312640008000130A30090303E
:100180008A018A20FE308A01022001308A01022081
:10019000FE308A0102200E308A0102200630B800AB
:1001A0008030B6005430AA002030AB00A901523094
:1001B000B000B1018A0173208A015220BA00CE300A
:1001C0003A07B200FF300318013EB30032088A013B
:1001D0000220BB0A64003B08103C8A110A12031D6E
:1001E000F728FE308A010220C0308A010220640014
:1001F0003B08203C8A110A12031D0B29FE308A019C
:10020000022001308A010220FE308A0102200230E1
:100210008A010220BB01FA308A0189208A01CE2896
:02400E00753DFE
:00000001FF
